
 Start         Length     Name                   Class
 0001:00000000 00015C3CH .text                   CODE
 0002:00000000 00000CB8H .data                   DATA
 0002:00000CB8 00000059H .bss                    BSS


Detailed map of segments

 0001:00000000 000000C6 C=CODE     S=.text    G=(none)   M=System   ACBP=A9
 0001:000000C8 000001EC C=CODE     S=.text    G=(none)   M=SysInit  ACBP=A9
 0001:000002B4 00000038 C=CODE     S=.text    G=(none)   M=Windows  ACBP=A9
 0001:000002EC 0000000E C=CODE     S=.text    G=(none)   M=Types    ACBP=A9
 0001:000002FC 0000000E C=CODE     S=.text    G=(none)   M=ActiveX  ACBP=A9
 0001:0000030C 00000038 C=CODE     S=.text    G=(none)   M=Messages ACBP=A9
 0001:00000344 00000046 C=CODE     S=.text    G=(none)   M=Classes  ACBP=A9
 0001:0000038C 0000000E C=CODE     S=.text    G=(none)   M=TypInfo  ACBP=A9
 0001:0000039C 0000000E C=CODE     S=.text    G=(none)   M=SysUtils ACBP=A9
 0001:000003AC 0000000E C=CODE     S=.text    G=(none)   M=SysConst ACBP=A9
 0001:000003BC 0000000E C=CODE     S=.text    G=(none)   M=Variants ACBP=A9
 0001:000003CC 0000000E C=CODE     S=.text    G=(none)   M=VarUtils ACBP=A9
 0001:000003DC 0000000E C=CODE     S=.text    G=(none)   M=RTLConsts ACBP=A9
 0001:000003EC 0000000E C=CODE     S=.text    G=(none)   M=Graphics ACBP=A9
 0001:000003FC 0000000E C=CODE     S=.text    G=(none)   M=Consts   ACBP=A9
 0001:0000040C 0000000E C=CODE     S=.text    G=(none)   M=OleServer ACBP=A9
 0001:0000041C 0000001E C=CODE     S=.text    G=(none)   M=ComObj   ACBP=A9
 0001:0000043C 0000000E C=CODE     S=.text    G=(none)   M=ComConst ACBP=A9
 0001:0000044C 00000186 C=CODE     S=.text    G=(none)   M=Controls ACBP=A9
 0001:000005D4 0000000E C=CODE     S=.text    G=(none)   M=ActnList ACBP=A9
 0001:000005E4 0000000E C=CODE     S=.text    G=(none)   M=Contnrs  ACBP=A9
 0001:000005F4 0000000E C=CODE     S=.text    G=(none)   M=Math     ACBP=A9
 0001:00000604 0000000E C=CODE     S=.text    G=(none)   M=ImgList  ACBP=A9
 0001:00000614 00000038 C=CODE     S=.text    G=(none)   M=CommCtrl ACBP=A9
 0001:0000064C 0000000E C=CODE     S=.text    G=(none)   M=Forms    ACBP=A9
 0001:0000065C 0000000E C=CODE     S=.text    G=(none)   M=HelpIntfs ACBP=A9
 0001:0000066C 0000000E C=CODE     S=.text    G=(none)   M=MultiMon ACBP=A9
 0001:0000067C 00000038 C=CODE     S=.text    G=(none)   M=Imm      ACBP=A9
 0001:000006B4 0000000E C=CODE     S=.text    G=(none)   M=Menus    ACBP=A9
 0001:000006C4 0000000E C=CODE     S=.text    G=(none)   M=WinHelpViewer ACBP=A9
 0001:000006D4 0000000E C=CODE     S=.text    G=(none)   M=StdActns ACBP=A9
 0001:000006E4 0000000E C=CODE     S=.text    G=(none)   M=Dialogs  ACBP=A9
 0001:000006F4 00000038 C=CODE     S=.text    G=(none)   M=ShlObj   ACBP=A9
 0001:0000072C 00000038 C=CODE     S=.text    G=(none)   M=UrlMon   ACBP=A9
 0001:00000764 00000038 C=CODE     S=.text    G=(none)   M=WinInet  ACBP=A9
 0001:0000079C 00000038 C=CODE     S=.text    G=(none)   M=RegStr   ACBP=A9
 0001:000007D4 00000038 C=CODE     S=.text    G=(none)   M=ShellAPI ACBP=A9
 0001:0000080C 0000000E C=CODE     S=.text    G=(none)   M=Printers ACBP=A9
 0001:0000081C 00000038 C=CODE     S=.text    G=(none)   M=WinSpool ACBP=A9
 0001:00000854 0000000E C=CODE     S=.text    G=(none)   M=StdCtrls ACBP=A9
 0001:00000864 00000038 C=CODE     S=.text    G=(none)   M=CommDlg  ACBP=A9
 0001:0000089C 00000038 C=CODE     S=.text    G=(none)   M=Dlgs     ACBP=A9
 0001:000008D4 0000000E C=CODE     S=.text    G=(none)   M=ExtCtrls ACBP=A9
 0001:000008E4 0000000E C=CODE     S=.text    G=(none)   M=StrUtils ACBP=A9
 0001:000008F4 0000000E C=CODE     S=.text    G=(none)   M=Clipbrd  ACBP=A9
 0001:00000904 0000000E C=CODE     S=.text    G=(none)   M=FlatSB   ACBP=A9
 0001:00000914 0000000E C=CODE     S=.text    G=(none)   M=OleConst ACBP=A9
 0001:00000924 0000011E C=CODE     S=.text    G=(none)   M=OleCtrls ACBP=A9
 0001:00000A44 0000000E C=CODE     S=.text    G=(none)   M=AxCtrls  ACBP=A9
 0001:00000A54 0000000E C=CODE     S=.text    G=(none)   M=StdVCL   ACBP=A9
 0001:00000A64 000031AC C=CODE     S=.text    G=(none)   M=Chartfx3 ACBP=A9
 0001:00003C10 00001B44 C=CODE     S=.text    G=(none)   M=VCSpell3 ACBP=A9
 0001:00005754 000077DC C=CODE     S=.text    G=(none)   M=VCF1     ACBP=A9
 0001:0000CF30 00008B24 C=CODE     S=.text    G=(none)   M=VCFI     ACBP=A9
 0001:00015A54 000001E5 C=CODE     S=.text    G=(none)   M=dclocx   ACBP=A9
 0002:00000000 00000028 C=DATA     S=.data    G=DGROUP   M=SysInit  ACBP=A9
 0002:00000028 00000184 C=DATA     S=.data    G=DGROUP   M=Chartfx3 ACBP=A9
 0002:000001AC 000000C0 C=DATA     S=.data    G=DGROUP   M=VCSpell3 ACBP=A9
 0002:0000026C 00000138 C=DATA     S=.data    G=DGROUP   M=VCF1     ACBP=A9
 0002:000003A4 00000914 C=DATA     S=.data    G=DGROUP   M=VCFI     ACBP=A9
 0002:00001000 00000018 C=BSS      S=.bss     G=DGROUP   M=SysInit  ACBP=A9
 0002:00001018 00000004 C=BSS      S=.bss     G=DGROUP   M=Windows  ACBP=A9
 0002:0000101C 00000004 C=BSS      S=.bss     G=DGROUP   M=Messages ACBP=A9
 0002:00001020 00000004 C=BSS      S=.bss     G=DGROUP   M=CommCtrl ACBP=A9
 0002:00001024 00000004 C=BSS      S=.bss     G=DGROUP   M=Imm      ACBP=A9
 0002:00001028 00000004 C=BSS      S=.bss     G=DGROUP   M=ShlObj   ACBP=A9
 0002:0000102C 00000004 C=BSS      S=.bss     G=DGROUP   M=UrlMon   ACBP=A9
 0002:00001030 00000004 C=BSS      S=.bss     G=DGROUP   M=WinInet  ACBP=A9
 0002:00001034 00000004 C=BSS      S=.bss     G=DGROUP   M=RegStr   ACBP=A9
 0002:00001038 00000004 C=BSS      S=.bss     G=DGROUP   M=ShellAPI ACBP=A9
 0002:0000103C 00000004 C=BSS      S=.bss     G=DGROUP   M=WinSpool ACBP=A9
 0002:00001040 00000004 C=BSS      S=.bss     G=DGROUP   M=CommDlg  ACBP=A9
 0002:00001044 00000004 C=BSS      S=.bss     G=DGROUP   M=Dlgs     ACBP=A9
 0002:00001048 00000004 C=BSS      S=.bss     G=DGROUP   M=Chartfx3 ACBP=A9
 0002:0000104C 00000004 C=BSS      S=.bss     G=DGROUP   M=VCSpell3 ACBP=A9
 0002:00001050 00000004 C=BSS      S=.bss     G=DGROUP   M=VCF1     ACBP=A9
 0002:00001054 00000004 C=BSS      S=.bss     G=DGROUP   M=VCFI     ACBP=A9


  Address         Publics by Name

 0002:00001034       .1
 0002:00001020       .1
 0002:00001038       .1
 0002:00001030       .1
 0002:00001028       .1
 0002:00001010       .1
 0002:00001024       .1
 0002:00001044       .1
 0002:0000101C       .1
 0002:00001040       .1
 0002:0000102C       .1
 0002:00001050       .2
 0002:00001048       .2
 0002:0000104C       .2
 0002:0000103C       .3
 0002:00001018       .3
 0002:00001054       .46
 0001:00015C14       @GetPackageInfoTable
 0001:00000200       @InitPkg
 0001:00015C1C       @PackageLoad
 0001:00000264       @PackageLoad
 0001:00015C28       @PackageUnload
 0001:00000270       @PackageUnload
 0001:00000100       AllocTlsBuffer
 0002:0000021C       CControlData
 0002:00000C64       CControlData
 0002:00000158       CControlData
 0002:00000350       CControlData
 0002:000002AC       CEventDispIDs
 0002:000001CC       CEventDispIDs
 0002:00000068       CEventDispIDs
 0002:00000BA4       CEventDispIDs
 0001:00003C08       Chartfx3
 0002:00000A54       CLASS_Attribute
 0002:00000B74       CLASS_Attributes
 0002:000008D4       CLASS_Axis
 0002:00000934       CLASS_AxisGrid
 0002:00000994       CLASS_AxisScale
 0002:000009D4       CLASS_AxisTitle
 0002:00000574       CLASS_Backdrop
 0002:000007D4       CLASS_Bar
 0002:000004B4       CLASS_Brush
 0002:000008F4       CLASS_CategoryScale
 0002:00000058       CLASS_Chartfx
 0002:00000A94       CLASS_Contour
 0002:00000B94       CLASS_ContourGradient
 0002:000003F4       CLASS_Coor
 0002:00000434       CLASS_Coor3
 0002:000006B4       CLASS_DataGrid
 0002:000008B4       CLASS_DataPoint
 0002:00000894       CLASS_DataPointLabel
 0002:00000AF4       CLASS_DataPoints
 0002:00000914       CLASS_DateScale
 0002:00000734       CLASS_Doughnut
 0002:00000A34       CLASS_Elevation
 0002:0000029C       CLASS_F1Book
 0002:000005F4       CLASS_Fill
 0002:00000654       CLASS_Footnote
 0002:00000594       CLASS_Frame
 0002:000005B4       CLASS_Gradient
 0002:000007F4       CLASS_HiLo
 0002:00000954       CLASS_Intersection
 0002:00000B14       CLASS_Labels
 0002:000009F4       CLASS_Label_
 0002:00000414       CLASS_LCoor
 0002:00000674       CLASS_Legend
 0002:00000A14       CLASS_Light
 0002:00000AB4       CLASS_LightSource
 0002:00000B54       CLASS_LightSources
 0002:00000534       CLASS_Location
 0002:00000454       CLASS_LRect
 0002:00000634       CLASS_Marker
 0002:00000614       CLASS_Pen
 0002:00000754       CLASS_Pie
 0002:000006D4       CLASS_Plot
 0002:00000714       CLASS_PlotBase
 0002:00000814       CLASS_Position
 0002:00000694       CLASS_PrintInformation
 0002:00000474       CLASS_Rect
 0002:000007B4       CLASS_Series
 0002:00000AD4       CLASS_SeriesCollection
 0002:00000854       CLASS_SeriesLabel
 0002:00000834       CLASS_SeriesMarker
 0002:000004D4       CLASS_Shadow
 0002:00000874       CLASS_StatLine
 0002:00000A74       CLASS_Surface
 0002:000004F4       CLASS_TextLayout
 0002:00000974       CLASS_Tick
 0002:00000514       CLASS_Title
 0002:000009B4       CLASS_ValueScale
 0002:000006F4       CLASS_View3d
 0002:000001BC       Class_VSSpell
 0002:000003D4       CLASS_VtChart
 0002:00000494       CLASS_VtColor
 0002:00000554       CLASS_VtFont
 0002:000005D4       CLASS_VtPicture
 0002:00000794       CLASS_Wall
 0002:00000774       CLASS_Weighting
 0002:00000B34       CLASS_XYZ
 0002:000000A8       CLicenseKey
 0002:000002F4       CLicenseKey
 0002:00000C08       CLicenseKey
 0002:000001F4       CLicenseKey
 0001:00015024       CoAttribute.Create
 0001:00015088       CoAttribute.CreateRemote
 0001:00015828       CoAttributes.Create
 0001:0001588C       CoAttributes.CreateRemote
 0001:00014574       CoAxis.Create
 0001:000145D8       CoAxis.CreateRemote
 0001:00014820       CoAxisGrid.Create
 0001:00014884       CoAxisGrid.CreateRemote
 0001:00014ACC       CoAxisScale.Create
 0001:00014B30       CoAxisScale.CreateRemote
 0001:00014C94       CoAxisTitle.Create
 0001:00014CF8       CoAxisTitle.CreateRemote
 0001:00012D68       CoBackdrop.Create
 0001:00012DCC       CoBackdrop.CreateRemote
 0001:00013E54       CoBar.Create
 0001:00013EB8       CoBar.CreateRemote
 0001:00012810       CoBrush.Create
 0001:00012874       CoBrush.CreateRemote
 0001:00014658       CoCategoryScale.Create
 0001:000146BC       CoCategoryScale.CreateRemote
 0001:000151EC       CoContour.Create
 0001:00015250       CoContour.CreateRemote
 0001:0001590C       CoContourGradient.Create
 0001:00015970       CoContourGradient.CreateRemote
 0001:000122B8       CoCoor.Create
 0001:0001231C       CoCoor.CreateRemote
 0001:00012480       CoCoor3.Create
 0001:000124E4       CoCoor3.CreateRemote
 0001:00013650       CoDataGrid.Create
 0001:000136B4       CoDataGrid.CreateRemote
 0001:00014490       CoDataPoint.Create
 0001:000144F4       CoDataPoint.CreateRemote
 0001:000143AC       CoDataPointLabel.Create
 0001:00014410       CoDataPointLabel.CreateRemote
 0001:00015498       CoDataPoints.Create
 0001:000154FC       CoDataPoints.CreateRemote
 0001:0001473C       CoDateScale.Create
 0001:000147A0       CoDateScale.CreateRemote
 0001:000139E0       CoDoughnut.Create
 0001:00013A44       CoDoughnut.CreateRemote
 0001:00014F40       CoElevation.Create
 0001:00014FA4       CoElevation.CreateRemote
 0001:000130F8       CoFill.Create
 0001:0001315C       CoFill.CreateRemote
 0001:000133A4       CoFootnote.Create
 0001:00013408       CoFootnote.CreateRemote
 0001:00012E4C       CoFrame.Create
 0001:00012EB0       CoFrame.CreateRemote
 0001:00012F30       CoGradient.Create
 0001:00012F94       CoGradient.CreateRemote
 0001:00013F38       CoHiLo.Create
 0001:00013F9C       CoHiLo.CreateRemote
 0001:00014904       CoIntersection.Create
 0001:00014968       CoIntersection.CreateRemote
 0001:0001557C       CoLabels.Create
 0001:000155E0       CoLabels.CreateRemote
 0001:00014D78       CoLabel_.Create
 0001:00014DDC       CoLabel_.CreateRemote
 0001:0001239C       CoLCoor.Create
 0001:00012400       CoLCoor.CreateRemote
 0001:00013488       CoLegend.Create
 0001:000134EC       CoLegend.CreateRemote
 0001:00014E5C       CoLight.Create
 0001:00014EC0       CoLight.CreateRemote
 0001:000152D0       CoLightSource.Create
 0001:00015334       CoLightSource.CreateRemote
 0001:00015744       CoLightSources.Create
 0001:000157A8       CoLightSources.CreateRemote
 0001:00012BA0       CoLocation.Create
 0001:00012C04       CoLocation.CreateRemote
 0001:00012564       CoLRect.Create
 0001:000125C8       CoLRect.CreateRemote
 0001:000132C0       CoMarker.Create
 0001:00013324       CoMarker.CreateRemote
 0001:00000644       CommCtrl
 0001:00000894       CommDlg
 0001:000131DC       CoPen.Create
 0001:00013240       CoPen.CreateRemote
 0001:00013AC4       CoPie.Create
 0001:00013B28       CoPie.CreateRemote
 0001:00013734       CoPlot.Create
 0001:00013798       CoPlot.CreateRemote
 0001:000138FC       CoPlotBase.Create
 0001:00013960       CoPlotBase.CreateRemote
 0001:0001401C       CoPosition.Create
 0001:00014080       CoPosition.CreateRemote
 0001:0001356C       CoPrintInformation.Create
 0001:000135D0       CoPrintInformation.CreateRemote
 0001:00012648       CoRect.Create
 0001:000126AC       CoRect.CreateRemote
 0001:00013D70       CoSeries.Create
 0001:00013DD4       CoSeries.CreateRemote
 0001:000153B4       CoSeriesCollection.Create
 0001:00015418       CoSeriesCollection.CreateRemote
 0001:000141E4       CoSeriesLabel.Create
 0001:00014248       CoSeriesLabel.CreateRemote
 0001:00014100       CoSeriesMarker.Create
 0001:00014164       CoSeriesMarker.CreateRemote
 0001:000128F4       CoShadow.Create
 0001:00012958       CoShadow.CreateRemote
 0001:000142C8       CoStatLine.Create
 0001:0001432C       CoStatLine.CreateRemote
 0001:00015108       CoSurface.Create
 0001:0001516C       CoSurface.CreateRemote
 0001:000129D8       CoTextLayout.Create
 0001:00012A3C       CoTextLayout.CreateRemote
 0001:000149E8       CoTick.Create
 0001:00014A4C       CoTick.CreateRemote
 0001:00012ABC       CoTitle.Create
 0001:00012B20       CoTitle.CreateRemote
 0001:00014BB0       CoValueScale.Create
 0001:00014C14       CoValueScale.CreateRemote
 0001:00013818       CoView3d.Create
 0001:0001387C       CoView3d.CreateRemote
 0001:0001272C       CoVtColor.Create
 0001:00012790       CoVtColor.CreateRemote
 0001:00012C84       CoVtFont.Create
 0001:00012CE8       CoVtFont.CreateRemote
 0001:00013014       CoVtPicture.Create
 0001:00013078       CoVtPicture.CreateRemote
 0001:00013C8C       CoWall.Create
 0001:00013CF0       CoWall.CreateRemote
 0001:00013BA8       CoWeighting.Create
 0001:00013C0C       CoWeighting.CreateRemote
 0001:00015660       CoXYZ.Create
 0001:000156C4       CoXYZ.CreateRemote
 0002:00000138       CTFontIDs
 0002:0000034C       CTPictureIDs
 0002:00000C60       CTPictureIDs
 0001:00015C34       dclocx
 0002:00000564       DIID_IBackdrop
 0002:000004A4       DIID_IBrush
 0002:00000484       DIID_IColor
 0002:000003E4       DIID_ICoor
 0002:00000424       DIID_ICoor3
 0002:000005E4       DIID_IFill
 0002:00000544       DIID_IFont
 0002:00000584       DIID_IFrame
 0002:000005A4       DIID_IGradient
 0002:00000404       DIID_ILCoor
 0002:00000524       DIID_ILocation
 0002:00000444       DIID_ILRect
 0002:000005C4       DIID_IPicture
 0002:00000464       DIID_IRect
 0002:000004C4       DIID_IShadow
 0002:000004E4       DIID_ITextLayout
 0002:00000A44       DIID_IVcAttribute
 0002:00000B64       DIID_IVcAttributes
 0002:000008C4       DIID_IVcAxis
 0002:00000924       DIID_IVcAxisGrid
 0002:000009C4       DIID_IVcAxisTitle
 0002:000007C4       DIID_IVcBar
 0002:000008E4       DIID_IVcCategoryScale
 0002:00000A84       DIID_IVcContour
 0002:00000B84       DIID_IVcContourGradient
 0002:000006A4       DIID_IVcDataGrid
 0002:000008A4       DIID_IVcDataPoint
 0002:00000884       DIID_IVcDataPointLabel
 0002:00000AE4       DIID_IVcDataPoints
 0002:00000904       DIID_IVcDateScale
 0002:00000724       DIID_IVcDoughnut
 0002:00000A24       DIID_IVcElevation
 0002:00000644       DIID_IVcFootnote
 0002:000007E4       DIID_IVcHiLo
 0002:00000944       DIID_IVcIntersection
 0002:000009E4       DIID_IVcLabel
 0002:00000B04       DIID_IVcLabels
 0002:00000664       DIID_IVcLegend
 0002:00000A04       DIID_IVcLight
 0002:00000AA4       DIID_IVcLightSource
 0002:00000B44       DIID_IVcLightSources
 0002:00000624       DIID_IVcMarker
 0002:00000604       DIID_IVcPen
 0002:00000744       DIID_IVcPie
 0002:000006C4       DIID_IVcPlot
 0002:00000704       DIID_IVcPlotBase
 0002:00000804       DIID_IVcPosition
 0002:00000684       DIID_IVcPrintInformation
 0002:00000984       DIID_IVcScale
 0002:000007A4       DIID_IVcSeries
 0002:00000AC4       DIID_IVcSeriesCollection
 0002:00000844       DIID_IVcSeriesLabel
 0002:00000824       DIID_IVcSeriesMarker
 0002:00000864       DIID_IVcStatLines
 0002:00000A64       DIID_IVcSurface
 0002:00000964       DIID_IVcTick
 0002:00000504       DIID_IVcTitle
 0002:000009A4       DIID_IVcValueScale
 0002:000006E4       DIID_IVcView3d
 0002:00000784       DIID_IVcWall
 0002:00000764       DIID_IVcWeighting
 0002:00000B24       DIID_IVcXYZ
 0002:00000038       DIID__DChartfx
 0002:00000048       DIID__DChartfxEvents
 0002:0000027C       DIID__DVCF1
 0002:0000028C       DIID__DVCF1Events
 0002:000003B4       DIID__DVtChart
 0002:000003C4       DIID__DVtChartEvents
 0001:000008CC       Dlgs
 0001:00011208       DoCreate
 0001:00001EC4       DoCreate
 0001:000073A0       DoCreate
 0001:000001AC       ExitProcessTLS
 0001:00000184       ExitThreadTLS
 0001:00015A1C       Finalization
 0001:0000027C       Finalization
 0001:000002B4       Finalization
 0001:0000030C       Finalization
 0001:00000614       Finalization
 0001:0000067C       Finalization
 0001:000006F4       Finalization
 0001:0000072C       Finalization
 0001:00000764       Finalization
 0001:0000079C       Finalization
 0001:000007D4       Finalization
 0001:00000864       Finalization
 0001:0000089C       Finalization
 0001:00003BD8       Finalization
 0001:0000571C       Finalization
 0001:0000CEF8       Finalization
 0001:0000081C       Finalization
 0001:000000C8       FreeLibrary
 0001:0000010C       GetTlsSize
 0002:0000100C       HInstance
 0001:000006AC       Imm
 0001:000001D0       InitializeModule
 0001:00000158       InitProcessTLS
 0001:00000114       InitThreadTLS
 0002:00000028       LIBID_ChartfxLib
 0002:0000026C       LIBID_VCIF1Lib
 0002:000003A4       LIBID_VCIFiLib
 0002:000001AC       LIBID_VspelocxLib
 0001:000000D0       LocalAlloc
 0001:000000D8       LocalFree
 0001:0000033C       Messages
 0002:00000000       Module
 0002:00001000       ModuleIsLib
 0002:00001001       ModuleIsPackage
 0001:000056F0       Register
 0001:00003BAC       Register
 0001:0000CECC       Register
 0001:000159F0       Register
 0001:000007CC       RegStr
 0001:00000804       ShellAPI
 0001:00000724       ShlObj
 0001:000002AC       SysInit
 0001:00003B50       TChartfx.AboutBox
 0001:00003380       TChartfx.CloseData
 0001:00003A94       TChartfx.CopyBitmap
 0001:00003A34       TChartfx.CopyData
 0001:00001F48       TChartfx.CreateControl
 0001:000033EC       TChartfx.DblClk
 0001:00003884       TChartfx.ExportFile
 0001:00001F68       TChartfx.GetControlInterface
 0001:000024C8       TChartfx.Get_Adm
 0001:000023F0       TChartfx.Get_BkColor
 0001:00002318       TChartfx.Get_Color
 0001:00002234       TChartfx.Get_Const_
 0001:00003234       TChartfx.Get_DecimalsNum
 0001:00002AAC       TChartfx.Get_FixLeg
 0001:00002684       TChartfx.Get_Fonts
 0001:00002ED4       TChartfx.Get_HFont
 0001:00002150       TChartfx.Get_IniValue
 0001:0000315C       TChartfx.Get_ItemColor
 0001:00003084       TChartfx.Get_ItemStyle
 0001:00002FAC       TChartfx.Get_ItemWidth
 0001:000029D8       TChartfx.Get_KeyLeg
 0001:00002C54       TChartfx.Get_KeySer
 0001:00002830       TChartfx.Get_Legend
 0001:000025AC       TChartfx.Get_Pattern
 0001:00002DFC       TChartfx.Get_RGBFont
 0001:00002904       TChartfx.Get_SerLeg
 0001:00002D28       TChartfx.Get_StatusText
 0001:0000275C       TChartfx.Get_Title
 0001:00001F88       TChartfx.Get_Value
 0001:0000206C       TChartfx.Get_XValue
 0001:00002B80       TChartfx.Get_YLeg
 0001:000038F0       TChartfx.ImportFile
 0001:00001EA8       TChartfx.InitControlData
 0001:00003818       TChartfx.Language
 0001:0000330C       TChartfx.OpenDataEx
 0001:00003710       TChartfx.Paint
 0001:000035AC       TChartfx.PrintIt
 0001:000039C8       TChartfx.ReadTemplate
 0001:00003AF4       TChartfx.Refresh
 0001:0000345C       TChartfx.RigClk
 0001:0000360C       TChartfx.Scroll
 0001:0000367C       TChartfx.SetStatusItem
 0001:0000379C       TChartfx.SetStripe
 0001:0000253C       TChartfx.Set_Adm
 0001:0000245C       TChartfx.Set_BkColor
 0001:00002384       TChartfx.Set_Color
 0001:000022A8       TChartfx.Set_Const_
 0001:000032A0       TChartfx.Set_DecimalsNum
 0001:00002B14       TChartfx.Set_FixLeg
 0001:000026F0       TChartfx.Set_Fonts
 0001:00002F40       TChartfx.Set_HFont
 0001:000021C4       TChartfx.Set_IniValue
 0001:000031C8       TChartfx.Set_ItemColor
 0001:000030F0       TChartfx.Set_ItemStyle
 0001:00003018       TChartfx.Set_ItemWidth
 0001:00002A40       TChartfx.Set_KeyLeg
 0001:00002CBC       TChartfx.Set_KeySer
 0001:00002898       TChartfx.Set_Legend
 0001:00002618       TChartfx.Set_Pattern
 0001:00002E68       TChartfx.Set_RGBFont
 0001:0000296C       TChartfx.Set_SerLeg
 0001:00002D90       TChartfx.Set_StatusText
 0001:000027C4       TChartfx.Set_Title
 0001:00001FFC       TChartfx.Set_Value
 0001:000020E0       TChartfx.Set_XValue
 0001:00002BE8       TChartfx.Set_YLeg
 0001:0000353C       TChartfx.ShowDialog
 0001:000034CC       TChartfx.Status
 0001:0000395C       TChartfx.WriteTemplate
 0001:0000CE70       TF1Book.AboutBox
 0001:00008FA0       TF1Book.AddColPageBreak
 0001:00009008       TF1Book.AddPageBreak
 0001:00009064       TF1Book.AddRowPageBreak
 0001:000090CC       TF1Book.AddSelection
 0001:00009140       TF1Book.Attach
 0001:000091A8       TF1Book.AttachToSS
 0001:0000CAA8       TF1Book.AutoFillItemsCount
 0001:00009210       TF1Book.CalculationDlg
 0001:0000926C       TF1Book.CancelEdit
 0001:000092C8       TF1Book.CheckRecalc
 0001:00009324       TF1Book.ClearClipboard
 0001:00009380       TF1Book.ClearRange
 0001:00009400       TF1Book.ColorPaletteDlg
 0001:0000945C       TF1Book.ColWidthDlg
 0001:000094B8       TF1Book.CopyAll
 0001:00009520       TF1Book.CopyRange
 0001:0000CB08       TF1Book.CopyRangeEx
 0001:00007424       TF1Book.CreateControl
 0001:0000C914       TF1Book.DefinedNameCount
 0001:000095B0       TF1Book.DefinedNameDlg
 0001:0000CC4C       TF1Book.DeleteAutoFillItems
 0001:0000960C       TF1Book.DeleteDefinedName
 0001:00009674       TF1Book.DeleteRange
 0001:0000C3C8       TF1Book.DeleteSheets
 0001:000096F4       TF1Book.Draw
 0001:00009798       TF1Book.EditClear
 0001:00009800       TF1Book.EditCopy
 0001:0000985C       TF1Book.EditCopyDown
 0001:000098B8       TF1Book.EditCopyRight
 0001:00009914       TF1Book.EditCut
 0001:00009970       TF1Book.EditDelete
 0001:0000C300       TF1Book.EditDeleteSheets
 0001:000099D8       TF1Book.EditInsert
 0001:0000C2A4       TF1Book.EditInsertSheets
 0001:00009A40       TF1Book.EditPaste
 0001:00008B5C       TF1Book.EditPasteValues
 0001:00009A9C       TF1Book.EndEdit
 0001:0000C840       TF1Book.ErrorNumberToText
 0001:00009AF8       TF1Book.FilePageSetupDlg
 0001:00009B54       TF1Book.FilePrint
 0001:00009BBC       TF1Book.FilePrintSetupDlg
 0001:00009C18       TF1Book.FormatAlignmentDlg
 0001:00009C74       TF1Book.FormatBorderDlg
 0001:00009CD0       TF1Book.FormatCurrency0
 0001:00009D2C       TF1Book.FormatCurrency2
 0001:00009D88       TF1Book.FormatDefaultFontDlg
 0001:00009DE4       TF1Book.FormatFixed
 0001:00009E40       TF1Book.FormatFixed2
 0001:00009E9C       TF1Book.FormatFontDlg
 0001:00009EF8       TF1Book.FormatFraction
 0001:00009F54       TF1Book.FormatGeneral
 0001:00009FB0       TF1Book.FormatHmmampm
 0001:0000A00C       TF1Book.FormatMdyy
 0001:0000A068       TF1Book.FormatNumberDlg
 0001:0000A0C4       TF1Book.FormatPatternDlg
 0001:0000A120       TF1Book.FormatPercent
 0001:0000C76C       TF1Book.FormatRCNr
 0001:0000A17C       TF1Book.FormatScientific
 0001:0000A1D8       TF1Book.GetActiveCell
 0001:00008BB8       TF1Book.GetAlignment
 0001:00008C2C       TF1Book.GetBorder
 0001:00007444       TF1Book.GetControlInterface
 0001:0000A244       TF1Book.GetDefaultFont
 0001:00008CBC       TF1Book.GetFont
 0001:0000A2B0       TF1Book.GetHdrSelection
 0001:0000A320       TF1Book.GetIteration
 0001:00008D4C       TF1Book.GetLineStyle
 0001:00008DBC       TF1Book.GetPattern
 0001:0000A390       TF1Book.GetPrintScale
 0001:00008E2C       TF1Book.GetProtection
 0001:0000A404       TF1Book.GetSelection
 0001:00008E98       TF1Book.GetTabbedText
 0001:0000CA3C       TF1Book.GetValidationRule
 0001:00008800       TF1Book.Get_AutoFillItems
 0001:000088D4       TF1Book.Get_ColHidden
 0001:00007464       TF1Book.Get_ColText
 0001:00007DEC       TF1Book.Get_ColWidth
 0001:0000821C       TF1Book.Get_ColWidthTwips
 0001:00007538       TF1Book.Get_DefinedName
 0001:00007F9C       TF1Book.Get_DefinedNameByIndex
 0001:0000760C       TF1Book.Get_EntryRC
 0001:000076EC       TF1Book.Get_FormattedTextRC
 0001:000077CC       TF1Book.Get_FormulaRC
 0001:000078AC       TF1Book.Get_LastColForRow
 0001:00007984       TF1Book.Get_LogicalRC
 0001:00007A68       TF1Book.Get_NumberRC
 0001:000082F4       TF1Book.Get_ObjItem
 0001:000083D4       TF1Book.Get_ObjItems
 0001:000084A8       TF1Book.Get_ObjName
 0001:0000857C       TF1Book.Get_ObjText
 0001:00008650       TF1Book.Get_ObjValue
 0001:00008728       TF1Book.Get_ObjVisible
 0001:00008144       TF1Book.Get_PaletteEntry
 0001:00007EC4       TF1Book.Get_RowHeight
 0001:000089AC       TF1Book.Get_RowHidden
 0001:00007B54       TF1Book.Get_RowText
 0001:00008070       TF1Book.Get_SheetName
 0001:00008A84       TF1Book.Get_SheetSelected
 0001:00007C28       TF1Book.Get_TextRC
 0001:00007D08       TF1Book.Get_TypeRC
 0001:0000A480       TF1Book.GotoDlg
 0001:0000A4DC       TF1Book.HeapMin
 0001:00007384       TF1Book.InitControlData
 0001:0000A538       TF1Book.InitTable
 0001:0000A594       TF1Book.InsertRange
 0001:0000C35C       TF1Book.InsertSheets
 0001:0000CE14       TF1Book.LaunchDesigner
 0001:0000A614       TF1Book.LineStyleDlg
 0001:0000A670       TF1Book.MoveRange
 0001:0000C490       TF1Book.NextColPageBreak
 0001:0000C4FC       TF1Book.NextRowPageBreak
 0001:0000A6F0       TF1Book.ObjAddItem
 0001:0000A75C       TF1Book.ObjAddSelection
 0001:0000A7C4       TF1Book.ObjBringToFront
 0001:0000A820       TF1Book.ObjDeleteItem
 0001:0000C568       TF1Book.ObjFirstID
 0001:0000A88C       TF1Book.ObjGetCell
 0001:0000C634       TF1Book.ObjGetItemCount
 0001:0000A900       TF1Book.ObjGetPos
 0001:0000A97C       TF1Book.ObjGetSelection
 0001:0000C70C       TF1Book.ObjGetSelectionCount
 0001:0000C6A0       TF1Book.ObjGetType
 0001:0000A9E8       TF1Book.ObjInsertItem
 0001:0000AA58       TF1Book.ObjNameDlg
 0001:0000C8A8       TF1Book.ObjNameToID
 0001:0000AAB4       TF1Book.ObjNew
 0001:0000AB30       TF1Book.ObjNewPicture
 0001:0000C5C8       TF1Book.ObjNextID
 0001:0000ABBC       TF1Book.ObjOptionsDlg
 0001:0000AC18       TF1Book.ObjPosToTwips
 0001:0000ACA4       TF1Book.ObjSendToBack
 0001:0000AD00       TF1Book.ObjSetCell
 0001:0000AD74       TF1Book.ObjSetPicture
 0001:0000ADF4       TF1Book.ObjSetPos
 0001:0000AE6C       TF1Book.ObjSetSelection
 0001:0000CCB4       TF1Book.ODBCConnect
 0001:0000CD24       TF1Book.ODBCDisconnect
 0001:0000CD80       TF1Book.ODBCQuery
 0001:0000AED4       TF1Book.OpenFileDlg
 0001:0000AF44       TF1Book.ProtectionDlg
 0001:0000AFA0       TF1Book.RangeToTwips
 0001:0000B030       TF1Book.Read
 0001:0000B09C       TF1Book.ReadFromBlob
 0001:0000B108       TF1Book.Recalc
 0001:0000C434       TF1Book.Refresh
 0001:0000B164       TF1Book.RemoveColPageBreak
 0001:0000B1CC       TF1Book.RemovePageBreak
 0001:0000B228       TF1Book.RemoveRowPageBreak
 0001:0000B290       TF1Book.RowHeightDlg
 0001:0000B2EC       TF1Book.SaveFileDlg
 0001:0000B35C       TF1Book.SaveWindowInfo
 0001:0000B3B8       TF1Book.SetActiveCell
 0001:0000B424       TF1Book.SetAlignment
 0001:0000B49C       TF1Book.SetBorder
 0001:0000C1B8       TF1Book.SetColHidden
 0001:0000B538       TF1Book.SetColWidth
 0001:0000B5B0       TF1Book.SetColWidthAuto
 0001:0000C22C       TF1Book.SetColWidthTwips
 0001:0000B630       TF1Book.SetDefaultFont
 0001:0000B69C       TF1Book.SetFont
 0001:0000B734       TF1Book.SetHdrSelection
 0001:0000B7A8       TF1Book.SetIteration
 0001:0000B81C       TF1Book.SetLineStyle
 0001:0000B890       TF1Book.SetPattern
 0001:0000B900       TF1Book.SetPrintAreaFromSelection
 0001:0000B95C       TF1Book.SetPrintScale
 0001:0000B9D4       TF1Book.SetPrintTitlesFromSelection
 0001:0000BA30       TF1Book.SetProtection
 0001:0000BA9C       TF1Book.SetRowHeight
 0001:0000BB14       TF1Book.SetRowHeightAuto
 0001:0000C144       TF1Book.SetRowHidden
 0001:0000BB94       TF1Book.SetSelection
 0001:00008F1C       TF1Book.SetTabbedText
 0001:0000C9D0       TF1Book.SetValidationRule
 0001:00008868       TF1Book.Set_AutoFillItems
 0001:00008940       TF1Book.Set_ColHidden
 0001:000074CC       TF1Book.Set_ColText
 0001:00007E58       TF1Book.Set_ColWidth
 0001:00008288       TF1Book.Set_ColWidthTwips
 0001:000075A0       TF1Book.Set_DefinedName
 0001:00008004       TF1Book.Set_DefinedNameByIndex
 0001:0000767C       TF1Book.Set_EntryRC
 0001:0000775C       TF1Book.Set_FormattedTextRC
 0001:0000783C       TF1Book.Set_FormulaRC
 0001:00007918       TF1Book.Set_LastColForRow
 0001:000079F4       TF1Book.Set_LogicalRC
 0001:00007AE0       TF1Book.Set_NumberRC
 0001:00008364       TF1Book.Set_ObjItem
 0001:0000843C       TF1Book.Set_ObjItems
 0001:00008510       TF1Book.Set_ObjName
 0001:000085E4       TF1Book.Set_ObjText
 0001:000086BC       TF1Book.Set_ObjValue
 0001:00008794       TF1Book.Set_ObjVisible
 0001:000081B0       TF1Book.Set_PaletteEntry
 0001:00007F30       TF1Book.Set_RowHeight
 0001:00008A18       TF1Book.Set_RowHidden
 0001:00007BBC       TF1Book.Set_RowText
 0001:000080D8       TF1Book.Set_SheetName
 0001:00008AF0       TF1Book.Set_SheetSelected
 0001:00007C98       TF1Book.Set_TextRC
 0001:00007D78       TF1Book.Set_TypeRC
 0001:0000BC08       TF1Book.ShowActiveCell
 0001:0000CBA0       TF1Book.Sort
 0001:0000BC64       TF1Book.Sort3
 0001:0000BCF0       TF1Book.SortDlg
 0001:0000C7E0       TF1Book.SS
 0001:0000BFB0       TF1Book.SSUpdate
 0001:0000C00C       TF1Book.SSVersion
 0001:0000BD4C       TF1Book.StartEdit
 0001:0000BDC0       TF1Book.SwapTables
 0001:0000BE28       TF1Book.TransactCommit
 0001:0000BE84       TF1Book.TransactRollback
 0001:0000BEE0       TF1Book.TransactStart
 0001:0000BF3C       TF1Book.TwipsToRC
 0001:0000C974       TF1Book.ValidationRuleDlg
 0001:0000C06C       TF1Book.Write
 0001:0000C0D8       TF1Book.WriteToBlob
 0001:000000E0       TlsAlloc
 0002:00001014       tlsBuffer
 0001:000000E8       TlsFree
 0001:000000F0       TlsGetValue
 0002:00001004       TlsIndex
 0002:AC9E9000       TlsLast
 0002:00000018       TlsProc
 0001:000000F8       TlsSetValue
 0001:00005090       TVSSpell.AboutBox
 0001:0000567C       TVSSpell.Get_CustomIsExtended
 0001:00005658       TVSSpell.Get_CustomIsReadOnly
 0001:00005268       TVSSpell.Get_CustomIsUpdateable
 0001:000053C8       TVSSpell.Get_DictionaryBlockCount
 0001:000053EC       TVSSpell.Get_DictionaryBlockSize
 0001:00005410       TVSSpell.Get_DictionaryCommonCount
 0001:00005434       TVSSpell.Get_DictionaryCompatibilityBits
 0001:00005458       TVSSpell.Get_DictionaryCopyright
 0001:00005488       TVSSpell.Get_DictionaryCopyrightDerived
 0001:000054B8       TVSSpell.Get_DictionaryFlags
 0001:00005150       TVSSpell.Get_DictionaryIsEnabled
 0001:000051C8       TVSSpell.Get_DictionaryIsLoaded
 0001:000050D8       TVSSpell.Get_DictionaryLanguage
 0001:000054DC       TVSSpell.Get_DictionaryLoadCount
 0001:00005500       TVSSpell.Get_DictionaryMakerVersion
 0001:000050FC       TVSSpell.Get_DictionaryName
 0001:00005174       TVSSpell.Get_DictionaryNameFull
 0001:00005524       TVSSpell.Get_DictionaryOpenCount
 0001:000051EC       TVSSpell.Get_DictionaryPerformance
 0001:000053A4       TVSSpell.Get_DictionaryPerformanceActual
 0001:0000512C       TVSSpell.Get_DictionaryStatus
 0001:00005548       TVSSpell.Get_DictionarySymbolSetSize
 0001:0000556C       TVSSpell.Get_DictionaryWordCount
 0001:000051A4       TVSSpell.Get_StandardIRListIsEnabled
 0001:00005238       TVSSpell.Get_Suggestion
 0001:00005058       TVSSpell.InitControlData
 0001:00005064       TVSSpell.InitControlInterface
 0001:000052B4       TVSSpell.Set_AddSuggestion
 0001:000052DC       TVSSpell.Set_AddToCustom
 0001:0000528C       TVSSpell.Set_AddToStandardIRList
 0001:00005304       TVSSpell.Set_ClearStandardIRList
 0001:0000532C       TVSSpell.Set_CloseDictionary
 0001:00005590       TVSSpell.Set_CreateCustomExtended
 0001:00005210       TVSSpell.Set_DictionaryPerformance
 0001:000055E0       TVSSpell.Set_EnableCustomUpdate
 0001:000055B8       TVSSpell.Set_EnableDictionary
 0001:000056A0       TVSSpell.Set_EnableStandardIRList
 0001:00005354       TVSSpell.Set_GetEntry
 0001:00005608       TVSSpell.Set_LoadDictionary
 0001:000056C8       TVSSpell.Set_OpenCustom
 0001:000050B0       TVSSpell.Set_OpenStandard
 0001:0000537C       TVSSpell.Set_RemoveFromStandardIRList
 0001:00005630       TVSSpell.Set_UnloadDictionary
 0001:0001225C       TVtChart.AboutBox
 0001:00011E8C       TVtChart.ActivateFormatMenu
 0001:00011990       TVtChart.ActivateSelectionDialog
 0001:00011F6C       TVtChart.CopyDataFromArray
 0001:00012014       TVtChart.CopyDataToArray
 0001:0001128C       TVtChart.CreateControl
 0001:000120BC       TVtChart.Draw
 0001:000121A4       TVtChart.EditChartData
 0001:00011934       TVtChart.EditCopy
 0001:000118D8       TVtChart.EditPaste
 0001:000112AC       TVtChart.GetControlInterface
 0001:00011C58       TVtChart.GetDLLVersion
 0001:00011EF8       TVtChart.GetMetafile
 0001:00011BDC       TVtChart.GetSelectedPart
 0001:0001145C       TVtChart.Get_Backdrop
 0001:000116B4       TVtChart.Get_DataGrid
 0001:00011394       TVtChart.Get_Footnote
 0001:00011844       TVtChart.Get_GetBitmap
 0001:000115EC       TVtChart.Get_Legend
 0001:0001177C       TVtChart.Get_Plot
 0001:00011524       TVtChart.Get_PrintInformation
 0001:000112CC       TVtChart.Get_Title
 0001:000111EC       TVtChart.InitControlData
 0001:000119EC       TVtChart.Layout
 0001:00011B00       TVtChart.PrintChart
 0001:00011AA4       TVtChart.PrintSetupDialog
 0001:00011D48       TVtChart.ReadFromFile
 0001:00012200       TVtChart.Refresh
 0001:00011B5C       TVtChart.SelectPart
 0001:000114BC       TVtChart.Set_Backdrop
 0001:00011714       TVtChart.Set_DataGrid
 0001:000113F4       TVtChart.Set_Footnote
 0001:0001164C       TVtChart.Set_Legend
 0001:000117DC       TVtChart.Set_Plot
 0001:00011584       TVtChart.Set_PrintInformation
 0001:0001132C       TVtChart.Set_Title
 0001:00011A48       TVtChart.ToDefaults
 0001:00011CC4       TVtChart.TwipsToChartPart
 0001:00012148       TVtChart.UseWizard
 0001:00011DB0       TVtChart.WritePictureToFile
 0001:00011E24       TVtChart.WriteToFile
 0001:000001DC       UninitializeModule
 0001:0000075C       UrlMon
 0001:0000CF28       VCF1
 0001:00015A4C       VCFI
 0001:0000574C       VCSpell3
 0001:000002E4       Windows
 0001:00000794       WinInet
 0001:0000084C       WinSpool


  Address         Publics by Value

 0002:AC9E9000       TlsLast
 0001:000000C8       FreeLibrary
 0001:000000D0       LocalAlloc
 0001:000000D8       LocalFree
 0001:000000E0       TlsAlloc
 0001:000000E8       TlsFree
 0001:000000F0       TlsGetValue
 0001:000000F8       TlsSetValue
 0001:00000100       AllocTlsBuffer
 0001:0000010C       GetTlsSize
 0001:00000114       InitThreadTLS
 0001:00000158       InitProcessTLS
 0001:00000184       ExitThreadTLS
 0001:000001AC       ExitProcessTLS
 0001:000001D0       InitializeModule
 0001:000001DC       UninitializeModule
 0001:00000200       @InitPkg
 0001:00000264       @PackageLoad
 0001:00000270       @PackageUnload
 0001:0000027C       Finalization
 0001:000002AC       SysInit
 0001:000002B4       Finalization
 0001:000002E4       Windows
 0001:0000030C       Finalization
 0001:0000033C       Messages
 0001:00000614       Finalization
 0001:00000644       CommCtrl
 0001:0000067C       Finalization
 0001:000006AC       Imm
 0001:000006F4       Finalization
 0001:00000724       ShlObj
 0001:0000072C       Finalization
 0001:0000075C       UrlMon
 0001:00000764       Finalization
 0001:00000794       WinInet
 0001:0000079C       Finalization
 0001:000007CC       RegStr
 0001:000007D4       Finalization
 0001:00000804       ShellAPI
 0001:0000081C       Finalization
 0001:0000084C       WinSpool
 0001:00000864       Finalization
 0001:00000894       CommDlg
 0001:0000089C       Finalization
 0001:000008CC       Dlgs
 0001:00001EA8       TChartfx.InitControlData
 0001:00001EC4       DoCreate
 0001:00001F48       TChartfx.CreateControl
 0001:00001F68       TChartfx.GetControlInterface
 0001:00001F88       TChartfx.Get_Value
 0001:00001FFC       TChartfx.Set_Value
 0001:0000206C       TChartfx.Get_XValue
 0001:000020E0       TChartfx.Set_XValue
 0001:00002150       TChartfx.Get_IniValue
 0001:000021C4       TChartfx.Set_IniValue
 0001:00002234       TChartfx.Get_Const_
 0001:000022A8       TChartfx.Set_Const_
 0001:00002318       TChartfx.Get_Color
 0001:00002384       TChartfx.Set_Color
 0001:000023F0       TChartfx.Get_BkColor
 0001:0000245C       TChartfx.Set_BkColor
 0001:000024C8       TChartfx.Get_Adm
 0001:0000253C       TChartfx.Set_Adm
 0001:000025AC       TChartfx.Get_Pattern
 0001:00002618       TChartfx.Set_Pattern
 0001:00002684       TChartfx.Get_Fonts
 0001:000026F0       TChartfx.Set_Fonts
 0001:0000275C       TChartfx.Get_Title
 0001:000027C4       TChartfx.Set_Title
 0001:00002830       TChartfx.Get_Legend
 0001:00002898       TChartfx.Set_Legend
 0001:00002904       TChartfx.Get_SerLeg
 0001:0000296C       TChartfx.Set_SerLeg
 0001:000029D8       TChartfx.Get_KeyLeg
 0001:00002A40       TChartfx.Set_KeyLeg
 0001:00002AAC       TChartfx.Get_FixLeg
 0001:00002B14       TChartfx.Set_FixLeg
 0001:00002B80       TChartfx.Get_YLeg
 0001:00002BE8       TChartfx.Set_YLeg
 0001:00002C54       TChartfx.Get_KeySer
 0001:00002CBC       TChartfx.Set_KeySer
 0001:00002D28       TChartfx.Get_StatusText
 0001:00002D90       TChartfx.Set_StatusText
 0001:00002DFC       TChartfx.Get_RGBFont
 0001:00002E68       TChartfx.Set_RGBFont
 0001:00002ED4       TChartfx.Get_HFont
 0001:00002F40       TChartfx.Set_HFont
 0001:00002FAC       TChartfx.Get_ItemWidth
 0001:00003018       TChartfx.Set_ItemWidth
 0001:00003084       TChartfx.Get_ItemStyle
 0001:000030F0       TChartfx.Set_ItemStyle
 0001:0000315C       TChartfx.Get_ItemColor
 0001:000031C8       TChartfx.Set_ItemColor
 0001:00003234       TChartfx.Get_DecimalsNum
 0001:000032A0       TChartfx.Set_DecimalsNum
 0001:0000330C       TChartfx.OpenDataEx
 0001:00003380       TChartfx.CloseData
 0001:000033EC       TChartfx.DblClk
 0001:0000345C       TChartfx.RigClk
 0001:000034CC       TChartfx.Status
 0001:0000353C       TChartfx.ShowDialog
 0001:000035AC       TChartfx.PrintIt
 0001:0000360C       TChartfx.Scroll
 0001:0000367C       TChartfx.SetStatusItem
 0001:00003710       TChartfx.Paint
 0001:0000379C       TChartfx.SetStripe
 0001:00003818       TChartfx.Language
 0001:00003884       TChartfx.ExportFile
 0001:000038F0       TChartfx.ImportFile
 0001:0000395C       TChartfx.WriteTemplate
 0001:000039C8       TChartfx.ReadTemplate
 0001:00003A34       TChartfx.CopyData
 0001:00003A94       TChartfx.CopyBitmap
 0001:00003AF4       TChartfx.Refresh
 0001:00003B50       TChartfx.AboutBox
 0001:00003BAC       Register
 0001:00003BD8       Finalization
 0001:00003C08       Chartfx3
 0001:00005058       TVSSpell.InitControlData
 0001:00005064       TVSSpell.InitControlInterface
 0001:00005090       TVSSpell.AboutBox
 0001:000050B0       TVSSpell.Set_OpenStandard
 0001:000050D8       TVSSpell.Get_DictionaryLanguage
 0001:000050FC       TVSSpell.Get_DictionaryName
 0001:0000512C       TVSSpell.Get_DictionaryStatus
 0001:00005150       TVSSpell.Get_DictionaryIsEnabled
 0001:00005174       TVSSpell.Get_DictionaryNameFull
 0001:000051A4       TVSSpell.Get_StandardIRListIsEnabled
 0001:000051C8       TVSSpell.Get_DictionaryIsLoaded
 0001:000051EC       TVSSpell.Get_DictionaryPerformance
 0001:00005210       TVSSpell.Set_DictionaryPerformance
 0001:00005238       TVSSpell.Get_Suggestion
 0001:00005268       TVSSpell.Get_CustomIsUpdateable
 0001:0000528C       TVSSpell.Set_AddToStandardIRList
 0001:000052B4       TVSSpell.Set_AddSuggestion
 0001:000052DC       TVSSpell.Set_AddToCustom
 0001:00005304       TVSSpell.Set_ClearStandardIRList
 0001:0000532C       TVSSpell.Set_CloseDictionary
 0001:00005354       TVSSpell.Set_GetEntry
 0001:0000537C       TVSSpell.Set_RemoveFromStandardIRList
 0001:000053A4       TVSSpell.Get_DictionaryPerformanceActual
 0001:000053C8       TVSSpell.Get_DictionaryBlockCount
 0001:000053EC       TVSSpell.Get_DictionaryBlockSize
 0001:00005410       TVSSpell.Get_DictionaryCommonCount
 0001:00005434       TVSSpell.Get_DictionaryCompatibilityBits
 0001:00005458       TVSSpell.Get_DictionaryCopyright
 0001:00005488       TVSSpell.Get_DictionaryCopyrightDerived
 0001:000054B8       TVSSpell.Get_DictionaryFlags
 0001:000054DC       TVSSpell.Get_DictionaryLoadCount
 0001:00005500       TVSSpell.Get_DictionaryMakerVersion
 0001:00005524       TVSSpell.Get_DictionaryOpenCount
 0001:00005548       TVSSpell.Get_DictionarySymbolSetSize
 0001:0000556C       TVSSpell.Get_DictionaryWordCount
 0001:00005590       TVSSpell.Set_CreateCustomExtended
 0001:000055B8       TVSSpell.Set_EnableDictionary
 0001:000055E0       TVSSpell.Set_EnableCustomUpdate
 0001:00005608       TVSSpell.Set_LoadDictionary
 0001:00005630       TVSSpell.Set_UnloadDictionary
 0001:00005658       TVSSpell.Get_CustomIsReadOnly
 0001:0000567C       TVSSpell.Get_CustomIsExtended
 0001:000056A0       TVSSpell.Set_EnableStandardIRList
 0001:000056C8       TVSSpell.Set_OpenCustom
 0001:000056F0       Register
 0001:0000571C       Finalization
 0001:0000574C       VCSpell3
 0001:00007384       TF1Book.InitControlData
 0001:000073A0       DoCreate
 0001:00007424       TF1Book.CreateControl
 0001:00007444       TF1Book.GetControlInterface
 0001:00007464       TF1Book.Get_ColText
 0001:000074CC       TF1Book.Set_ColText
 0001:00007538       TF1Book.Get_DefinedName
 0001:000075A0       TF1Book.Set_DefinedName
 0001:0000760C       TF1Book.Get_EntryRC
 0001:0000767C       TF1Book.Set_EntryRC
 0001:000076EC       TF1Book.Get_FormattedTextRC
 0001:0000775C       TF1Book.Set_FormattedTextRC
 0001:000077CC       TF1Book.Get_FormulaRC
 0001:0000783C       TF1Book.Set_FormulaRC
 0001:000078AC       TF1Book.Get_LastColForRow
 0001:00007918       TF1Book.Set_LastColForRow
 0001:00007984       TF1Book.Get_LogicalRC
 0001:000079F4       TF1Book.Set_LogicalRC
 0001:00007A68       TF1Book.Get_NumberRC
 0001:00007AE0       TF1Book.Set_NumberRC
 0001:00007B54       TF1Book.Get_RowText
 0001:00007BBC       TF1Book.Set_RowText
 0001:00007C28       TF1Book.Get_TextRC
 0001:00007C98       TF1Book.Set_TextRC
 0001:00007D08       TF1Book.Get_TypeRC
 0001:00007D78       TF1Book.Set_TypeRC
 0001:00007DEC       TF1Book.Get_ColWidth
 0001:00007E58       TF1Book.Set_ColWidth
 0001:00007EC4       TF1Book.Get_RowHeight
 0001:00007F30       TF1Book.Set_RowHeight
 0001:00007F9C       TF1Book.Get_DefinedNameByIndex
 0001:00008004       TF1Book.Set_DefinedNameByIndex
 0001:00008070       TF1Book.Get_SheetName
 0001:000080D8       TF1Book.Set_SheetName
 0001:00008144       TF1Book.Get_PaletteEntry
 0001:000081B0       TF1Book.Set_PaletteEntry
 0001:0000821C       TF1Book.Get_ColWidthTwips
 0001:00008288       TF1Book.Set_ColWidthTwips
 0001:000082F4       TF1Book.Get_ObjItem
 0001:00008364       TF1Book.Set_ObjItem
 0001:000083D4       TF1Book.Get_ObjItems
 0001:0000843C       TF1Book.Set_ObjItems
 0001:000084A8       TF1Book.Get_ObjName
 0001:00008510       TF1Book.Set_ObjName
 0001:0000857C       TF1Book.Get_ObjText
 0001:000085E4       TF1Book.Set_ObjText
 0001:00008650       TF1Book.Get_ObjValue
 0001:000086BC       TF1Book.Set_ObjValue
 0001:00008728       TF1Book.Get_ObjVisible
 0001:00008794       TF1Book.Set_ObjVisible
 0001:00008800       TF1Book.Get_AutoFillItems
 0001:00008868       TF1Book.Set_AutoFillItems
 0001:000088D4       TF1Book.Get_ColHidden
 0001:00008940       TF1Book.Set_ColHidden
 0001:000089AC       TF1Book.Get_RowHidden
 0001:00008A18       TF1Book.Set_RowHidden
 0001:00008A84       TF1Book.Get_SheetSelected
 0001:00008AF0       TF1Book.Set_SheetSelected
 0001:00008B5C       TF1Book.EditPasteValues
 0001:00008BB8       TF1Book.GetAlignment
 0001:00008C2C       TF1Book.GetBorder
 0001:00008CBC       TF1Book.GetFont
 0001:00008D4C       TF1Book.GetLineStyle
 0001:00008DBC       TF1Book.GetPattern
 0001:00008E2C       TF1Book.GetProtection
 0001:00008E98       TF1Book.GetTabbedText
 0001:00008F1C       TF1Book.SetTabbedText
 0001:00008FA0       TF1Book.AddColPageBreak
 0001:00009008       TF1Book.AddPageBreak
 0001:00009064       TF1Book.AddRowPageBreak
 0001:000090CC       TF1Book.AddSelection
 0001:00009140       TF1Book.Attach
 0001:000091A8       TF1Book.AttachToSS
 0001:00009210       TF1Book.CalculationDlg
 0001:0000926C       TF1Book.CancelEdit
 0001:000092C8       TF1Book.CheckRecalc
 0001:00009324       TF1Book.ClearClipboard
 0001:00009380       TF1Book.ClearRange
 0001:00009400       TF1Book.ColorPaletteDlg
 0001:0000945C       TF1Book.ColWidthDlg
 0001:000094B8       TF1Book.CopyAll
 0001:00009520       TF1Book.CopyRange
 0001:000095B0       TF1Book.DefinedNameDlg
 0001:0000960C       TF1Book.DeleteDefinedName
 0001:00009674       TF1Book.DeleteRange
 0001:000096F4       TF1Book.Draw
 0001:00009798       TF1Book.EditClear
 0001:00009800       TF1Book.EditCopy
 0001:0000985C       TF1Book.EditCopyDown
 0001:000098B8       TF1Book.EditCopyRight
 0001:00009914       TF1Book.EditCut
 0001:00009970       TF1Book.EditDelete
 0001:000099D8       TF1Book.EditInsert
 0001:00009A40       TF1Book.EditPaste
 0001:00009A9C       TF1Book.EndEdit
 0001:00009AF8       TF1Book.FilePageSetupDlg
 0001:00009B54       TF1Book.FilePrint
 0001:00009BBC       TF1Book.FilePrintSetupDlg
 0001:00009C18       TF1Book.FormatAlignmentDlg
 0001:00009C74       TF1Book.FormatBorderDlg
 0001:00009CD0       TF1Book.FormatCurrency0
 0001:00009D2C       TF1Book.FormatCurrency2
 0001:00009D88       TF1Book.FormatDefaultFontDlg
 0001:00009DE4       TF1Book.FormatFixed
 0001:00009E40       TF1Book.FormatFixed2
 0001:00009E9C       TF1Book.FormatFontDlg
 0001:00009EF8       TF1Book.FormatFraction
 0001:00009F54       TF1Book.FormatGeneral
 0001:00009FB0       TF1Book.FormatHmmampm
 0001:0000A00C       TF1Book.FormatMdyy
 0001:0000A068       TF1Book.FormatNumberDlg
 0001:0000A0C4       TF1Book.FormatPatternDlg
 0001:0000A120       TF1Book.FormatPercent
 0001:0000A17C       TF1Book.FormatScientific
 0001:0000A1D8       TF1Book.GetActiveCell
 0001:0000A244       TF1Book.GetDefaultFont
 0001:0000A2B0       TF1Book.GetHdrSelection
 0001:0000A320       TF1Book.GetIteration
 0001:0000A390       TF1Book.GetPrintScale
 0001:0000A404       TF1Book.GetSelection
 0001:0000A480       TF1Book.GotoDlg
 0001:0000A4DC       TF1Book.HeapMin
 0001:0000A538       TF1Book.InitTable
 0001:0000A594       TF1Book.InsertRange
 0001:0000A614       TF1Book.LineStyleDlg
 0001:0000A670       TF1Book.MoveRange
 0001:0000A6F0       TF1Book.ObjAddItem
 0001:0000A75C       TF1Book.ObjAddSelection
 0001:0000A7C4       TF1Book.ObjBringToFront
 0001:0000A820       TF1Book.ObjDeleteItem
 0001:0000A88C       TF1Book.ObjGetCell
 0001:0000A900       TF1Book.ObjGetPos
 0001:0000A97C       TF1Book.ObjGetSelection
 0001:0000A9E8       TF1Book.ObjInsertItem
 0001:0000AA58       TF1Book.ObjNameDlg
 0001:0000AAB4       TF1Book.ObjNew
 0001:0000AB30       TF1Book.ObjNewPicture
 0001:0000ABBC       TF1Book.ObjOptionsDlg
 0001:0000AC18       TF1Book.ObjPosToTwips
 0001:0000ACA4       TF1Book.ObjSendToBack
 0001:0000AD00       TF1Book.ObjSetCell
 0001:0000AD74       TF1Book.ObjSetPicture
 0001:0000ADF4       TF1Book.ObjSetPos
 0001:0000AE6C       TF1Book.ObjSetSelection
 0001:0000AED4       TF1Book.OpenFileDlg
 0001:0000AF44       TF1Book.ProtectionDlg
 0001:0000AFA0       TF1Book.RangeToTwips
 0001:0000B030       TF1Book.Read
 0001:0000B09C       TF1Book.ReadFromBlob
 0001:0000B108       TF1Book.Recalc
 0001:0000B164       TF1Book.RemoveColPageBreak
 0001:0000B1CC       TF1Book.RemovePageBreak
 0001:0000B228       TF1Book.RemoveRowPageBreak
 0001:0000B290       TF1Book.RowHeightDlg
 0001:0000B2EC       TF1Book.SaveFileDlg
 0001:0000B35C       TF1Book.SaveWindowInfo
 0001:0000B3B8       TF1Book.SetActiveCell
 0001:0000B424       TF1Book.SetAlignment
 0001:0000B49C       TF1Book.SetBorder
 0001:0000B538       TF1Book.SetColWidth
 0001:0000B5B0       TF1Book.SetColWidthAuto
 0001:0000B630       TF1Book.SetDefaultFont
 0001:0000B69C       TF1Book.SetFont
 0001:0000B734       TF1Book.SetHdrSelection
 0001:0000B7A8       TF1Book.SetIteration
 0001:0000B81C       TF1Book.SetLineStyle
 0001:0000B890       TF1Book.SetPattern
 0001:0000B900       TF1Book.SetPrintAreaFromSelection
 0001:0000B95C       TF1Book.SetPrintScale
 0001:0000B9D4       TF1Book.SetPrintTitlesFromSelection
 0001:0000BA30       TF1Book.SetProtection
 0001:0000BA9C       TF1Book.SetRowHeight
 0001:0000BB14       TF1Book.SetRowHeightAuto
 0001:0000BB94       TF1Book.SetSelection
 0001:0000BC08       TF1Book.ShowActiveCell
 0001:0000BC64       TF1Book.Sort3
 0001:0000BCF0       TF1Book.SortDlg
 0001:0000BD4C       TF1Book.StartEdit
 0001:0000BDC0       TF1Book.SwapTables
 0001:0000BE28       TF1Book.TransactCommit
 0001:0000BE84       TF1Book.TransactRollback
 0001:0000BEE0       TF1Book.TransactStart
 0001:0000BF3C       TF1Book.TwipsToRC
 0001:0000BFB0       TF1Book.SSUpdate
 0001:0000C00C       TF1Book.SSVersion
 0001:0000C06C       TF1Book.Write
 0001:0000C0D8       TF1Book.WriteToBlob
 0001:0000C144       TF1Book.SetRowHidden
 0001:0000C1B8       TF1Book.SetColHidden
 0001:0000C22C       TF1Book.SetColWidthTwips
 0001:0000C2A4       TF1Book.EditInsertSheets
 0001:0000C300       TF1Book.EditDeleteSheets
 0001:0000C35C       TF1Book.InsertSheets
 0001:0000C3C8       TF1Book.DeleteSheets
 0001:0000C434       TF1Book.Refresh
 0001:0000C490       TF1Book.NextColPageBreak
 0001:0000C4FC       TF1Book.NextRowPageBreak
 0001:0000C568       TF1Book.ObjFirstID
 0001:0000C5C8       TF1Book.ObjNextID
 0001:0000C634       TF1Book.ObjGetItemCount
 0001:0000C6A0       TF1Book.ObjGetType
 0001:0000C70C       TF1Book.ObjGetSelectionCount
 0001:0000C76C       TF1Book.FormatRCNr
 0001:0000C7E0       TF1Book.SS
 0001:0000C840       TF1Book.ErrorNumberToText
 0001:0000C8A8       TF1Book.ObjNameToID
 0001:0000C914       TF1Book.DefinedNameCount
 0001:0000C974       TF1Book.ValidationRuleDlg
 0001:0000C9D0       TF1Book.SetValidationRule
 0001:0000CA3C       TF1Book.GetValidationRule
 0001:0000CAA8       TF1Book.AutoFillItemsCount
 0001:0000CB08       TF1Book.CopyRangeEx
 0001:0000CBA0       TF1Book.Sort
 0001:0000CC4C       TF1Book.DeleteAutoFillItems
 0001:0000CCB4       TF1Book.ODBCConnect
 0001:0000CD24       TF1Book.ODBCDisconnect
 0001:0000CD80       TF1Book.ODBCQuery
 0001:0000CE14       TF1Book.LaunchDesigner
 0001:0000CE70       TF1Book.AboutBox
 0001:0000CECC       Register
 0001:0000CEF8       Finalization
 0001:0000CF28       VCF1
 0001:000111EC       TVtChart.InitControlData
 0001:00011208       DoCreate
 0001:0001128C       TVtChart.CreateControl
 0001:000112AC       TVtChart.GetControlInterface
 0001:000112CC       TVtChart.Get_Title
 0001:0001132C       TVtChart.Set_Title
 0001:00011394       TVtChart.Get_Footnote
 0001:000113F4       TVtChart.Set_Footnote
 0001:0001145C       TVtChart.Get_Backdrop
 0001:000114BC       TVtChart.Set_Backdrop
 0001:00011524       TVtChart.Get_PrintInformation
 0001:00011584       TVtChart.Set_PrintInformation
 0001:000115EC       TVtChart.Get_Legend
 0001:0001164C       TVtChart.Set_Legend
 0001:000116B4       TVtChart.Get_DataGrid
 0001:00011714       TVtChart.Set_DataGrid
 0001:0001177C       TVtChart.Get_Plot
 0001:000117DC       TVtChart.Set_Plot
 0001:00011844       TVtChart.Get_GetBitmap
 0001:000118D8       TVtChart.EditPaste
 0001:00011934       TVtChart.EditCopy
 0001:00011990       TVtChart.ActivateSelectionDialog
 0001:000119EC       TVtChart.Layout
 0001:00011A48       TVtChart.ToDefaults
 0001:00011AA4       TVtChart.PrintSetupDialog
 0001:00011B00       TVtChart.PrintChart
 0001:00011B5C       TVtChart.SelectPart
 0001:00011BDC       TVtChart.GetSelectedPart
 0001:00011C58       TVtChart.GetDLLVersion
 0001:00011CC4       TVtChart.TwipsToChartPart
 0001:00011D48       TVtChart.ReadFromFile
 0001:00011DB0       TVtChart.WritePictureToFile
 0001:00011E24       TVtChart.WriteToFile
 0001:00011E8C       TVtChart.ActivateFormatMenu
 0001:00011EF8       TVtChart.GetMetafile
 0001:00011F6C       TVtChart.CopyDataFromArray
 0001:00012014       TVtChart.CopyDataToArray
 0001:000120BC       TVtChart.Draw
 0001:00012148       TVtChart.UseWizard
 0001:000121A4       TVtChart.EditChartData
 0001:00012200       TVtChart.Refresh
 0001:0001225C       TVtChart.AboutBox
 0001:000122B8       CoCoor.Create
 0001:0001231C       CoCoor.CreateRemote
 0001:0001239C       CoLCoor.Create
 0001:00012400       CoLCoor.CreateRemote
 0001:00012480       CoCoor3.Create
 0001:000124E4       CoCoor3.CreateRemote
 0001:00012564       CoLRect.Create
 0001:000125C8       CoLRect.CreateRemote
 0001:00012648       CoRect.Create
 0001:000126AC       CoRect.CreateRemote
 0001:0001272C       CoVtColor.Create
 0001:00012790       CoVtColor.CreateRemote
 0001:00012810       CoBrush.Create
 0001:00012874       CoBrush.CreateRemote
 0001:000128F4       CoShadow.Create
 0001:00012958       CoShadow.CreateRemote
 0001:000129D8       CoTextLayout.Create
 0001:00012A3C       CoTextLayout.CreateRemote
 0001:00012ABC       CoTitle.Create
 0001:00012B20       CoTitle.CreateRemote
 0001:00012BA0       CoLocation.Create
 0001:00012C04       CoLocation.CreateRemote
 0001:00012C84       CoVtFont.Create
 0001:00012CE8       CoVtFont.CreateRemote
 0001:00012D68       CoBackdrop.Create
 0001:00012DCC       CoBackdrop.CreateRemote
 0001:00012E4C       CoFrame.Create
 0001:00012EB0       CoFrame.CreateRemote
 0001:00012F30       CoGradient.Create
 0001:00012F94       CoGradient.CreateRemote
 0001:00013014       CoVtPicture.Create
 0001:00013078       CoVtPicture.CreateRemote
 0001:000130F8       CoFill.Create
 0001:0001315C       CoFill.CreateRemote
 0001:000131DC       CoPen.Create
 0001:00013240       CoPen.CreateRemote
 0001:000132C0       CoMarker.Create
 0001:00013324       CoMarker.CreateRemote
 0001:000133A4       CoFootnote.Create
 0001:00013408       CoFootnote.CreateRemote
 0001:00013488       CoLegend.Create
 0001:000134EC       CoLegend.CreateRemote
 0001:0001356C       CoPrintInformation.Create
 0001:000135D0       CoPrintInformation.CreateRemote
 0001:00013650       CoDataGrid.Create
 0001:000136B4       CoDataGrid.CreateRemote
 0001:00013734       CoPlot.Create
 0001:00013798       CoPlot.CreateRemote
 0001:00013818       CoView3d.Create
 0001:0001387C       CoView3d.CreateRemote
 0001:000138FC       CoPlotBase.Create
 0001:00013960       CoPlotBase.CreateRemote
 0001:000139E0       CoDoughnut.Create
 0001:00013A44       CoDoughnut.CreateRemote
 0001:00013AC4       CoPie.Create
 0001:00013B28       CoPie.CreateRemote
 0001:00013BA8       CoWeighting.Create
 0001:00013C0C       CoWeighting.CreateRemote
 0001:00013C8C       CoWall.Create
 0001:00013CF0       CoWall.CreateRemote
 0001:00013D70       CoSeries.Create
 0001:00013DD4       CoSeries.CreateRemote
 0001:00013E54       CoBar.Create
 0001:00013EB8       CoBar.CreateRemote
 0001:00013F38       CoHiLo.Create
 0001:00013F9C       CoHiLo.CreateRemote
 0001:0001401C       CoPosition.Create
 0001:00014080       CoPosition.CreateRemote
 0001:00014100       CoSeriesMarker.Create
 0001:00014164       CoSeriesMarker.CreateRemote
 0001:000141E4       CoSeriesLabel.Create
 0001:00014248       CoSeriesLabel.CreateRemote
 0001:000142C8       CoStatLine.Create
 0001:0001432C       CoStatLine.CreateRemote
 0001:000143AC       CoDataPointLabel.Create
 0001:00014410       CoDataPointLabel.CreateRemote
 0001:00014490       CoDataPoint.Create
 0001:000144F4       CoDataPoint.CreateRemote
 0001:00014574       CoAxis.Create
 0001:000145D8       CoAxis.CreateRemote
 0001:00014658       CoCategoryScale.Create
 0001:000146BC       CoCategoryScale.CreateRemote
 0001:0001473C       CoDateScale.Create
 0001:000147A0       CoDateScale.CreateRemote
 0001:00014820       CoAxisGrid.Create
 0001:00014884       CoAxisGrid.CreateRemote
 0001:00014904       CoIntersection.Create
 0001:00014968       CoIntersection.CreateRemote
 0001:000149E8       CoTick.Create
 0001:00014A4C       CoTick.CreateRemote
 0001:00014ACC       CoAxisScale.Create
 0001:00014B30       CoAxisScale.CreateRemote
 0001:00014BB0       CoValueScale.Create
 0001:00014C14       CoValueScale.CreateRemote
 0001:00014C94       CoAxisTitle.Create
 0001:00014CF8       CoAxisTitle.CreateRemote
 0001:00014D78       CoLabel_.Create
 0001:00014DDC       CoLabel_.CreateRemote
 0001:00014E5C       CoLight.Create
 0001:00014EC0       CoLight.CreateRemote
 0001:00014F40       CoElevation.Create
 0001:00014FA4       CoElevation.CreateRemote
 0001:00015024       CoAttribute.Create
 0001:00015088       CoAttribute.CreateRemote
 0001:00015108       CoSurface.Create
 0001:0001516C       CoSurface.CreateRemote
 0001:000151EC       CoContour.Create
 0001:00015250       CoContour.CreateRemote
 0001:000152D0       CoLightSource.Create
 0001:00015334       CoLightSource.CreateRemote
 0001:000153B4       CoSeriesCollection.Create
 0001:00015418       CoSeriesCollection.CreateRemote
 0001:00015498       CoDataPoints.Create
 0001:000154FC       CoDataPoints.CreateRemote
 0001:0001557C       CoLabels.Create
 0001:000155E0       CoLabels.CreateRemote
 0001:00015660       CoXYZ.Create
 0001:000156C4       CoXYZ.CreateRemote
 0001:00015744       CoLightSources.Create
 0001:000157A8       CoLightSources.CreateRemote
 0001:00015828       CoAttributes.Create
 0001:0001588C       CoAttributes.CreateRemote
 0001:0001590C       CoContourGradient.Create
 0001:00015970       CoContourGradient.CreateRemote
 0001:000159F0       Register
 0001:00015A1C       Finalization
 0001:00015A4C       VCFI
 0001:00015C14       @GetPackageInfoTable
 0001:00015C1C       @PackageLoad
 0001:00015C28       @PackageUnload
 0001:00015C34       dclocx
 0002:00000000       Module
 0002:00000018       TlsProc
 0002:00000028       LIBID_ChartfxLib
 0002:00000038       DIID__DChartfx
 0002:00000048       DIID__DChartfxEvents
 0002:00000058       CLASS_Chartfx
 0002:00000068       CEventDispIDs
 0002:000000A8       CLicenseKey
 0002:00000138       CTFontIDs
 0002:00000158       CControlData
 0002:000001AC       LIBID_VspelocxLib
 0002:000001BC       Class_VSSpell
 0002:000001CC       CEventDispIDs
 0002:000001F4       CLicenseKey
 0002:0000021C       CControlData
 0002:0000026C       LIBID_VCIF1Lib
 0002:0000027C       DIID__DVCF1
 0002:0000028C       DIID__DVCF1Events
 0002:0000029C       CLASS_F1Book
 0002:000002AC       CEventDispIDs
 0002:000002F4       CLicenseKey
 0002:0000034C       CTPictureIDs
 0002:00000350       CControlData
 0002:000003A4       LIBID_VCIFiLib
 0002:000003B4       DIID__DVtChart
 0002:000003C4       DIID__DVtChartEvents
 0002:000003D4       CLASS_VtChart
 0002:000003E4       DIID_ICoor
 0002:000003F4       CLASS_Coor
 0002:00000404       DIID_ILCoor
 0002:00000414       CLASS_LCoor
 0002:00000424       DIID_ICoor3
 0002:00000434       CLASS_Coor3
 0002:00000444       DIID_ILRect
 0002:00000454       CLASS_LRect
 0002:00000464       DIID_IRect
 0002:00000474       CLASS_Rect
 0002:00000484       DIID_IColor
 0002:00000494       CLASS_VtColor
 0002:000004A4       DIID_IBrush
 0002:000004B4       CLASS_Brush
 0002:000004C4       DIID_IShadow
 0002:000004D4       CLASS_Shadow
 0002:000004E4       DIID_ITextLayout
 0002:000004F4       CLASS_TextLayout
 0002:00000504       DIID_IVcTitle
 0002:00000514       CLASS_Title
 0002:00000524       DIID_ILocation
 0002:00000534       CLASS_Location
 0002:00000544       DIID_IFont
 0002:00000554       CLASS_VtFont
 0002:00000564       DIID_IBackdrop
 0002:00000574       CLASS_Backdrop
 0002:00000584       DIID_IFrame
 0002:00000594       CLASS_Frame
 0002:000005A4       DIID_IGradient
 0002:000005B4       CLASS_Gradient
 0002:000005C4       DIID_IPicture
 0002:000005D4       CLASS_VtPicture
 0002:000005E4       DIID_IFill
 0002:000005F4       CLASS_Fill
 0002:00000604       DIID_IVcPen
 0002:00000614       CLASS_Pen
 0002:00000624       DIID_IVcMarker
 0002:00000634       CLASS_Marker
 0002:00000644       DIID_IVcFootnote
 0002:00000654       CLASS_Footnote
 0002:00000664       DIID_IVcLegend
 0002:00000674       CLASS_Legend
 0002:00000684       DIID_IVcPrintInformation
 0002:00000694       CLASS_PrintInformation
 0002:000006A4       DIID_IVcDataGrid
 0002:000006B4       CLASS_DataGrid
 0002:000006C4       DIID_IVcPlot
 0002:000006D4       CLASS_Plot
 0002:000006E4       DIID_IVcView3d
 0002:000006F4       CLASS_View3d
 0002:00000704       DIID_IVcPlotBase
 0002:00000714       CLASS_PlotBase
 0002:00000724       DIID_IVcDoughnut
 0002:00000734       CLASS_Doughnut
 0002:00000744       DIID_IVcPie
 0002:00000754       CLASS_Pie
 0002:00000764       DIID_IVcWeighting
 0002:00000774       CLASS_Weighting
 0002:00000784       DIID_IVcWall
 0002:00000794       CLASS_Wall
 0002:000007A4       DIID_IVcSeries
 0002:000007B4       CLASS_Series
 0002:000007C4       DIID_IVcBar
 0002:000007D4       CLASS_Bar
 0002:000007E4       DIID_IVcHiLo
 0002:000007F4       CLASS_HiLo
 0002:00000804       DIID_IVcPosition
 0002:00000814       CLASS_Position
 0002:00000824       DIID_IVcSeriesMarker
 0002:00000834       CLASS_SeriesMarker
 0002:00000844       DIID_IVcSeriesLabel
 0002:00000854       CLASS_SeriesLabel
 0002:00000864       DIID_IVcStatLines
 0002:00000874       CLASS_StatLine
 0002:00000884       DIID_IVcDataPointLabel
 0002:00000894       CLASS_DataPointLabel
 0002:000008A4       DIID_IVcDataPoint
 0002:000008B4       CLASS_DataPoint
 0002:000008C4       DIID_IVcAxis
 0002:000008D4       CLASS_Axis
 0002:000008E4       DIID_IVcCategoryScale
 0002:000008F4       CLASS_CategoryScale
 0002:00000904       DIID_IVcDateScale
 0002:00000914       CLASS_DateScale
 0002:00000924       DIID_IVcAxisGrid
 0002:00000934       CLASS_AxisGrid
 0002:00000944       DIID_IVcIntersection
 0002:00000954       CLASS_Intersection
 0002:00000964       DIID_IVcTick
 0002:00000974       CLASS_Tick
 0002:00000984       DIID_IVcScale
 0002:00000994       CLASS_AxisScale
 0002:000009A4       DIID_IVcValueScale
 0002:000009B4       CLASS_ValueScale
 0002:000009C4       DIID_IVcAxisTitle
 0002:000009D4       CLASS_AxisTitle
 0002:000009E4       DIID_IVcLabel
 0002:000009F4       CLASS_Label_
 0002:00000A04       DIID_IVcLight
 0002:00000A14       CLASS_Light
 0002:00000A24       DIID_IVcElevation
 0002:00000A34       CLASS_Elevation
 0002:00000A44       DIID_IVcAttribute
 0002:00000A54       CLASS_Attribute
 0002:00000A64       DIID_IVcSurface
 0002:00000A74       CLASS_Surface
 0002:00000A84       DIID_IVcContour
 0002:00000A94       CLASS_Contour
 0002:00000AA4       DIID_IVcLightSource
 0002:00000AB4       CLASS_LightSource
 0002:00000AC4       DIID_IVcSeriesCollection
 0002:00000AD4       CLASS_SeriesCollection
 0002:00000AE4       DIID_IVcDataPoints
 0002:00000AF4       CLASS_DataPoints
 0002:00000B04       DIID_IVcLabels
 0002:00000B14       CLASS_Labels
 0002:00000B24       DIID_IVcXYZ
 0002:00000B34       CLASS_XYZ
 0002:00000B44       DIID_IVcLightSources
 0002:00000B54       CLASS_LightSources
 0002:00000B64       DIID_IVcAttributes
 0002:00000B74       CLASS_Attributes
 0002:00000B84       DIID_IVcContourGradient
 0002:00000B94       CLASS_ContourGradient
 0002:00000BA4       CEventDispIDs
 0002:00000C08       CLicenseKey
 0002:00000C60       CTPictureIDs
 0002:00000C64       CControlData
 0002:00001000       ModuleIsLib
 0002:00001001       ModuleIsPackage
 0002:00001004       TlsIndex
 0002:0000100C       HInstance
 0002:00001010       .1
 0002:00001014       tlsBuffer
 0002:00001018       .3
 0002:0000101C       .1
 0002:00001020       .1
 0002:00001024       .1
 0002:00001028       .1
 0002:0000102C       .1
 0002:00001030       .1
 0002:00001034       .1
 0002:00001038       .1
 0002:0000103C       .3
 0002:00001040       .1
 0002:00001044       .1
 0002:00001048       .2
 0002:0000104C       .2
 0002:00001050       .2
 0002:00001054       .46


Bound resource files

dclocx.res
chartfx.dcr
vcspell.dcr
vcfrmla1.dcr
vcfimprs.dcr
C:\TEMP\dtf29CF.tmp


Program entry point at 0001:00015C34
